:100000000C9400070C9444070C9444070C94440788
:100010000C9444070C9444070C9444070C94440734
:100020000C9444070C9444070C945D120C942F1309
:100030000C9444070C9444070C9444070C94440714
:100040000C9444070C94072C0C9444070C9444071C
:100050000C9444070C940E220C9444070C9444070F
:100060000C9444070C9444070C9444070C944407E4
:100070000C9444070C9444070C9444070C944407D4
:100080000C9444070C9444070C9444070C944407C4
:100090000C9444070C9444070C9444070C944407B4
:1000A0000C9444070C9444070C9444079413B6131F
:1000B000A114B613A114F8131B14A1147014831403
:1000C000D117D117FF17FF1742187E187F1A7F1A12
:1000D00096187F1A8D198D19591A7F1A7F1A6D1A61
:1000E0000000F0A123024C003900E100648100000F
:1000F0001E00140004001D0031714D001F001A0085
:1001000016001B002E002A00200008000700060031
:1001100038002C00210015000900190030004A00A9
:10012000220017000A00050000006574AE000154AB
:100130000000007F0000E300AB00025400000077E5
:100140000000E20023001C000B00110000002971D8
:10015000240018000D00100050004B0025000C007A
:100160000E00360051002800260012000F00370054
:1001700052002B0027001300330038714F004E004F
:100180002D002F003482E500C100000001000100B5
:1001900001000100010000003A001E0231002202AD
:1001A000010001003B001414210235000100010090
:1001B0003C00241425022514010001003D002714F1
:1001C00026022614010001003E0064142E023014A1
:1001D000000001000100010000000100000001001A
:1001E0000100010000000100000001003F0052007A
:1001F00051002302000001004000240021001E00E5
:10020000010001004100250022001F00370001000D
:100210004200260023002000270001004300300296
:1002200030002D14270201004400450001000100A8
:1002300001000000010001000100010001000000B8
:100240003A000100F700FB00010001003B00F40050
:10025000F200FA00FD00F5003C00F000F100F900AA
:10026000FE00F4003D00F500F300FC00FF0001007B
:100270003E000100F800F60000000100010001004E
:100280000000010000000100010001000000010069
:10029000000001003F0001000100B4000000010067
:1002A0004000AA00AC00B600010001004100A80017
:1002B000AD00B5000100B7004200A900AE00B900D2
:1002C0000100B60043000100AB00B70001000100CF
:1002D0004400450001000100010000000A00253033
:1002E000313662003A200025303258000A722F63FE
:1002F0002030313233343536373839414243444582
:10030000460A000A002530325800626F756E636538
:10031000213A20006C6566742073696465206174FD
:100320007461636865640A006C656674207369644F
:1003300065206E6F7420726573706F6E64696E678E
:100340000A00747279696E6720746F207265736534
:1003500074206D637032333031380A000A444542EC
:1003600055473A20656E61626C65642E0A005B73C6
:100370005D004B6579626F617264207374617274A1
:100380002E0A005B575D005B535D005B525D005BB6
:10039000445D005B435D0016034500720067006F1B
:1003A0000044006F007800200045005A000000164D
:1003B000034500720067006F0044006F0078002062
:1003C0000045005A0000000403090409028D0005DD
:1003D0000100A0FA09040000010301010009211134
:1003E000010001223F000705810308000A090401FA
:1003F000000103010200092111010001224D000743
:1004000005820308000A0904020001030000000934
:1004100021110100012236000705830308000A09A3
:100420000403000203000000092111010001222041
:1004300000070584032000010705040320000109CB
:100440000404000103000000092111010001223908
:1004500000070585031000011201100100000008CB
:10046000EDFE071301000102000105010906A101CB
:10047000050719E029E71500250195087501810296
:100480000508190129059505750191029501750366
:100490009101050719002977150025019578750147
:1004A0008102C00631FF0974A1010975150025FFFD
:1004B0009520750881020976150025FF952075089D
:1004C0009102C005010980A101850216010026B72D
:1004D000001A01002AB700751095018100C0050CB3
:1004E0000901A1018503160100269C021A01002AB8
:1004F0009C02751095018100C005010902A1010946
:1005000001A10005091901290515002501950575A9
:100510000181029501750381010501093009311539
:1005200081257F95027508810609381581257F95FB
:100530000175088106050C0A38021581257F950191
:1005400075088106C0C005010906A101050719E06B
:1005500029E71500250195087501810295017508A7
:10056000810105081901290595057501910295017B
:10057000750391010507190029FF150025FF950650
:1005800075088100C00A002530325820006B65795B
:10059000626F6172645F7265706F72743A20000AF4
:1005A0000025303258006B6579626F6172645F7349
:1005B00065745F6C65643A200064656C5F6B657997
:1005C0005F6269743A2063616E27742064656C3AD7
:1005D00020253032580A006164645F6B65795F6280
:1005E00069743A2063616E2774206164643A20253F
:1005F0003032580A00646F6E652E0A00626F6F67B2
:100600006D61676963207363616E3A202E2E2E2020
:1006100000290A002575002F002575005D2800259A
:10062000640020002564002000256400200025646B
:10063000007C0025303258006D6F7573656B6579ED
:10064000205B62746E7C782079207620685D287249
:1006500065702F61636C293A205B006D6B5F776872
:1006600065656C5F74696D655F746F5F6D6178203F
:100670003D2025640A006D6B5F776865656C5F6D72
:1006800061785F7370656564203D2025640A006DA4
:100690006B5F74696D655F746F5F6D6178203D207D
:1006A00025640A006D6B5F6D61785F7370656564CA
:1006B000203D2025640A006D6B5F696E746572765B
:1006C000616C203D2025640A006D6B5F64656C6180
:1006D00079203D2025640A006D6B5F776865656C45
:1006E0005F74696D655F746F5F6D6178203D202573
:1006F000640A006D6B5F776865656C5F6D61785F3C
:100700007370656564203D2025640A006D6B5F741D
:10071000696D655F746F5F6D6178203D2025640AA7
:10072000006D6B5F6D61785F7370656564203D205F
:1007300025640A006D6B5F696E74657276616C206A
:100740003D2025640A006D6B5F64656C6179203D16
:100750002025640A000A00257500363A207768656E
:10076000656C5F74696D655F746F5F6D61783A2069
:10077000000A00257500353A20776865656C5F6D65
:1007800061785F73706565643A20000A0025750022
:10079000343A2074696D655F746F5F6D61783A20DB
:1007A000000A00257500333A206D61785F7370652B
:1007B00065643A20000A00257500323A20696E749B
:1007C000657276616C286D73293A20000A002575E0
:1007D00000313A2064656C6179282A31306D7329C3
:1007E0003A20000A092D2056616C756573202D0A88
:1007F000004D3E004D25643E20003F00736574208F
:1008000064656661756C740A00433E200077686514
:1008100072652064656C74613A20637572736F72DF
:100820003D25642C20776865656C3D25640A536519
:100830006520687474703A2F2F656E2E77696B6926
:1008400070656469612E6F72672F77696B692F4DD0
:100850006F7573655F6B6579730A000A092D204D0A
:100860006F7573656B6579202D0A4553432F713A77
:1008700009717569740A313A0964656C6179282ACD
:1008800031306D73290A323A09696E746572766186
:100890006C286D73290A333A096D61785F7370654E
:1008A00065640A343A0974696D655F746F5F6D61E0
:1008B000780A353A09776865656C5F6D61785F73B2
:1008C000706565640A363A09776865656C5F7469B6
:1008D0006D655F746F5F6D61780A0A703A097072B6
:1008E000696E742076616C7565730A643A09736584
:1008F000742064656661756C74730A75703A092BAF
:10090000310A646F776E3A092D310A706775703A53
:10091000092B31300A7067646F776E3A092D3130D8
:100920000A0A7370656564203D2064656C746120FB
:100930002A206D61785F7370656564202A202872B3
:100940006570656174202F2074696D655F746F5FD9
:100950006D6178290A003F004D3E2000433E200093
:100960004C25640A000A092D20436F6E736F6C6575
:10097000202D0A4553432F713A09717569740A6D28
:100980003A096D6F7573656B65790A000A092D2048
:100990004D61676963202D0A643A09646562756771
:1009A0000A783A096465627567206D6174726978C6
:1009B0000A6B3A096465627567206B6579626F61DD
:1009C00072640A6D3A096465627567206D6F7573AC
:1009D000650A763A0976657273696F6E0A733A0929
:1009E0007374617475730A633A09636F6E736F6C25
:1009F00065206D6F64650A302D343A096C61796544
:100A000072302D34284631302D4634290A50617514
:100A1000733A09626F6F746C6F616465720A653A4C
:100A200009656570726F6D0A6E3A094E4B524F0A36
:100A30007A3A09736C656570204C4544207465737F
:100A4000740A000A002575002E6E6B726F3A200042
:100A50000A002575002E737761705F6261636B73A6
:100A60006C6173685F6261636B73706163653A2088
:100A7000000A002575002E737761705F67726176DA
:100A8000655F6573633A20000A002575002E6E6F5E
:100A90005F6775693A20000A002575002E7377613B
:100AA000705F72616C745F726775693A20000A004A
:100AB0002575002E737761705F6C616C745F6C6775
:100AC00075693A20000A002575002E636170736C09
:100AD0006F636B5F746F5F636F6E74726F6C3A20DD
:100AE000000A002575002E737761705F636F6E7466
:100AF000726F6C5F636170736C6F636B3A20000A96
:100B00000025303258006B65796D61705F636F6EE0
:100B10006669672E7261773A20000A002575002EFB
:100B20006D6F7573653A20000A002575002E6B65A0
:100B300079626F6172643A20000A002575002E6D9B
:100B400061747269783A20000A002575002E656E7E
:100B500061626C653A20000A0025303258006465F5
:100B60006275675F636F6E6669672E7261773A20A0
:100B7000000A0025750064656661756C745F6C61C0
:100B80007965723A20003F004E4B524F3A206F6613
:100B9000660A004E4B524F3A206F6E0A0074696D20
:100BA00065725F636F756E743A202530346C580A35
:100BB000006B6579626F6172645F6E6B726F3A2071
:100BC00025580A006B6579626F6172645F69646CB5
:100BD000653A2025580A006B6579626F6172645F1F
:100BE00070726F746F636F6C3A2025580A00686FDB
:100BF00073745F6B6579626F6172645F6C65647357
:100C000028293A2025580A000A092D2053746174B6
:100C10007573202D0A004743433A20342E382E3274
:100C2000204156522D4C4942433A20312E382E3025
:100C3000204156525F415243483A20617672350A4C
:100C4000004F5054494F4E533A204C554641204294
:100C50004F4F544D41474943204D4F5553454B4508
:100C6000592045585452414B455920434F4E534FFC
:100C70004C4520434F4D4D414E44204E4B524F204A
:100C80003531320A004255494C443A203932323526
:100C9000343532202830353A33363A3335204A61FC
:100CA0006E2032302032303136290A005649443A1B
:100CB00020307846454544284572676F446F782058
:100CC000455A29205049443A20307831333037286A
:100CD0004572676F446F7820455A29205645523A2D
:100CE000203078303030310A00444553433A207484
:100CF0002E6D2E6B2E206B6579626F61726420669B
:100D000069726D7761726520666F72204572676FD8
:100D1000646F780A000A092D2056657273696F6E38
:100D2000202D0A000A6D6F7573653A206F66660A9A
:100D3000000A6D6F7573653A206F6E0A000A6B6565
:100D400079626F6172643A206F66660A000A6B65A9
:100D500079626F6172643A206F6E0A000A6D617485
:100D60007269783A206F66660A000A6D617472696A
:100D7000783A206F6E0A000A64656275673A206FE0
:100D80006E0A000A64656275673A206F66660A003B
:100D90000A0A626F6F746C6F616465722E2E2E206A
:100DA00000433E20006565636F6E6669673A0A001E
:100DB000536C656570204C454420746573740A005B
:100DC0000000000000000000000000010204060A0C
:100DD0000F17202C3A4A5D71879DB3C7DAE9F5FCFD
:100DE000FFFCF5E9DAC7B39D87715D4A3A2C2017FD
:100DF0000F0A0604020100000000000000000000CD
:100E000011241FBECFEFDAE0DEBFCDBF04B603FE74
:100E100024C08091F9019091FA01A091FB01B09159
:100E2000FC018730904BA740B04BB9F41092F90108
:100E30001092FA011092FB011092FC0114BE84B7CB
:100E4000877F84BF88E10FB6F8948093600010928A
:100E500060000FBEE0E0FFE3099511E0A0E0B1E023
:100E6000EAEAFBE502C005900D92AA33B107D9F773
:100E700011E0AAE3B1E001C01D92A93FB107E1F77B
:100E80000E94970F0C94D32D0C940000FF93EF93C6
:100E9000E0913A01F0913B01309709F00995EF910B
:100EA000FF910895FC018591803011F0EFDFFBCFB9
:100EB0000895FF27E0E230E247FF0CC0419597FF1D
:100EC00009C0EDE26095709580959095611D711D4A
:100ED000811D911D27FF02C0219530E350E2AA2712
:100EE000660F771F881F991FAA1FA41710F0A41B55
:100EF00063955A95A9F7AA3008F0A95FA05DAF9352
:100F0000F395611571058105910541F7ED3211F4F5
:100F1000EF93F395F21718F43F93F395FBCF8F916E
:100F2000B5DFFA95E1F70895E991F991859180305F
:100F300021F0853219F0AADFF9CF089520E0E89476
:100F400055915532C1F3503311F4689455915A3389
:100F500048F4505390F3220F022E220F220F200D3F
:100F6000250FF4CF0EF4219589919991533619F3F9
:100F7000533729F1533559F1BC0188279927E89453
:100F80005C3621F48991999168945591543639F4DD
:100F900046EF7EF077FF0DC08FEF9FEF0AC0553709
:100FA0004AE039F0583540E121F0523642E009F08C
:100FB0000895FF93EF937DDFEF91FF91B7CFFF93FC
:100FC000EF93FC0181918030B9F360DFFBCFFF9399
:100FD000EF9368DFF1CFDF93CF93CDB7DEB72596E0
:100FE000A3DFCF91DF91089561110BC0FC018281D5
:100FF000882321F085EE0E94651603C085EE0E94CD
:101000002D1780E090E0089508956091BC017091E3
:10101000BD018091BE019091BF010E94122156989E
:101020005E9825982D9826982E9827982F9881308D
:1010300029F0823031F4269A2E9A0895259A2D9A15
:10104000089556985E98089585E098E0892B11F0F0
:101050000E94050880E090E0089556985E982598D3
:101060002D9826982E9827982F988FEF90E09093A0
:1010700089008093880090938B0080938A009093DE
:101080008D0080938C00259A2D9A2FEF80E792E0B7
:10109000215080409040E1F700C00000269A2E9A2F
:1010A0002FEF80E792E0215080409040E1F700C0B0
:1010B0000000279A2F9A2FEF80E792E0215080407E
:1010C0009040E1F700C0000025982D982FEF80E7B1
:1010D00092E0215080409040E1F700C00000269847
:1010E0002E982FEF80E792E0215080409040E1F76A
:1010F00000C0000027982F9856985E9825982D9844
:1011000026982E9827982F98089589EA8093800032
:1011100089E08093810024982C983F988AB18F743D
:101120008AB96E98479A8BB1806B8BB9769A0E9478
:101130002D0884E098E0892B11F00E94040880E0DB
:1011400090E0089580E28093000180913C0181113C
:101150000EC00E94F10881E080933C012FEF83EDE7
:1011600090E3215080409040E1F700C0000080E40F
:101170000E94F7088093000181112EC00E9421096E
:1011800080930001811128C00E94210980930001F1
:10119000811122C08FE30E942109809300018111F7
:1011A0001BC00E94190980E40E94F7088093000187
:1011B000811112C08CE00E942109809300018111ED
:1011C0000BC00E94210980930001811105C08FE3AB
:1011D0000E942109809300010E9419098091000159
:1011E00008951092B9008AE08093B800089594EAB7
:1011F0009093BC009091BC0097FFFCCF9091B900F8
:10120000987F983021F0903111F081E0089580931B
:10121000BB0084E88093BC008091BC0087FFFCCFBA
:101220008091B900887F883111F0803471F780E0B7
:10123000089584E98093BC008091BC0084FDFCCFBC
:1012400008958093BB0084E88093BC008091BC002B
:1012500087FFFCCF9091B900987F81E0983209F424
:1012600080E0089584E88093BC008091BC0087FFF3
:10127000FCCF8091BB00089580910001811115C0C1
:1012800080E40E94F7088093000181110CC082E184
:101290000E94210980930001811105C08FEF0E94F7
:1012A0002109809300010E94190984B1807F84B9CB
:1012B00085B1807F85B98AB1837F8AB98BB1837FFD
:1012C0008BB93E98469808950E94A2088093000129
:1012D0000E943C0980B38C7080BB81B3836F81BB5B
:1012E000ECE4F1E0AEE3B1E011921D9281E0EA3569
:1012F000F807D1F785E898E0892B11F00C94850860
:1013000008959F92AF92BF92CF92DF92EF92FF9299
:101310000F931F93CF93DF93809100018823E1F017
:1013200080913D018F5F80933D01811115C082E462
:1013300093E00E9452070E94A20880930001882334
:1013400029F088E293E00E94520706C084E193E00E
:101350000E9452070E942D080EE311E0C0E0D0E089
:10136000BB24B39482E0A82ECC24C394D12C25E0D6
:10137000E22E23E0F22EC73000F5809100018111AA
:1013800062C080E40E94F70880930001811112C0BE
:1013900082E10E9421098093000181110BC0C601E6
:1013A0000C2E01C0880F0A94EAF780950E9421094B
:1013B000809300010E94190946C0CA30A1F028F4A8
:1013C000C83059F0C93061F005C0CC3089F070F0F8
:1013D000CD3089F0209A289810C0219A29980DC004
:1013E000229A2A980AC0239A2B9807C0529A01C0C1
:1013F000539A5B9802C03E9A4698E0EAEA95F1F764
:101400008FB1799985C092E081708B25892B7C9B67
:1014100002C090E001C094E0892B7D9B02C090E067
:1014200001C098E0892B7E9B02C090E001C090E152
:10143000892B9FB19095991F9927991F9295990F84
:10144000907E892B10C080910001811176C080E4CC
:101450000E94F70880930001882309F45BC0912C57
:101460000E941909892DF8019081981739F180831C
:1014700080910101882301F18091D70180FF04C090
:101480008AE093E00E9452078091D70180FF0CC050
:10149000809101011F928F93FF92EF920E94EB07C0
:1014A0000F900F900F900F908091D70180FF04C094
:1014B00083E093E00E945207A09201010E943C0940
:1014C00021960F5F1F4FCE30D10509F054CF809188
:1014D00001018823B1F0815080930101882339F004
:1014E0008FE99FE00197F1F700C000000AC0ACE46B
:1014F000B1E0EEE3F1E081918D9391E0EC34F907F6
:10150000D1F784E298E0892BD1F00E94240817C01B
:1015100090E07ACF83E10E9421098093000181113C
:101520009ECF81E40E94F70880930001811197CF3C
:101530000E943209982E909493CF80E094CF81E05E
:10154000DF91CF911F910F91FF90EF90DF90CF909F
:10155000BF90AF909F900895E82FF0E0E45BFE4FBE
:1015600080810895CF92DF92EF92FF920F931F93A5
:10157000CF93DF938CEE92E00E9452073CE4E32E7F
:1015800031E0F32EC0E0D0E047EEC42E42E0D42E8E
:101590000EED12E0DF93CF93DF92CF920E94EB0724
:1015A00084EE92E00E945207F70181917F0190E062
:1015B0000E9477219F938F931F930F930E94EB07B5
:1015C0008CED92E00E94520721968DB79EB7089647
:1015D0000FB6F8949EBF0FBE8DBFCE30D105D1F6A9
:1015E000DF91CF911F910F91FF90EF90DF90CF90FF
:1015F00008958B3B910578F4883A910540F5853A3A
:101600009105D0F48430910508F0B1C08130910586
:1016100009F4ADC06BC0803E910508F467C0883EF8
:10162000910508F4A4C09C01205F310920313105E7
:1016300008F05CC090650895853A910509F459C099
:10164000863A910509F458C083E890E40895883AF1
:10165000910509F454C0893A910509F453C08A3AB6
:10166000910509F452C08B3A910509F451C08C3AA6
:10167000910509F450C08D3A910509F44FC0803BA3
:10168000910509F44EC08E3A910509F44DC08F3A88
:10169000910509F44CC0813B910509F44BC0823B94
:1016A000910509F44AC0833B910509F449C0843B84
:1016B000910509F448C0853B910509F447C0863B74
:1016C000910509F446C0873B910509F445C0883B64
:1016D000910509F444C0893B910509F443C08A3B54
:1016E000910509F042C08AE296E4089580E090E016
:1016F000089581E890E4089582E890E4089582EEE8
:1017000094E4089589EE94E408958AEE94E40895AB
:1017100085EB94E4089586EB94E4089587EB94E4D4
:1017200008958CEC94E408958DEC94E4089583E896
:1017300095E408958AE895E4089582E995E408958A
:1017400084E995E4089581E296E4089583E296E4BD
:10175000089584E296E4089585E296E4089586E289
:1017600096E4089587E296E4089580E094E408956D
:10177000089596E0799FF001112494E5899FE00D8A
:10178000F11D1124E60FF11DEE0FFF1FEC51FF4F6D
:10179000859194910895880F991F805A9040FC017B
:1017A000859194910895880F991F80529F4FFC0155
:1017B00085919491089526E0729FF001112444E5EB
:1017C000849FE00DF11D1124E60FF11DEE0FFF1FA8
:1017D000EC51FF4F25913491C9019A9581159F4194
:1017E00010F4C9010895C90190528115904128F45F
:1017F000C9019F700E94D30B0895C90190538115B0
:10180000904120F4C9019927906C0895211580E535
:10181000380769F40E94A01A9FEF24E34CE091502E
:1018200020404040E1F700C000000C9433222130FA
:1018300080E5380751F48CE593E00E9452078091CF
:10184000D70181608093D7010895C9019055811512
:10185000904108F050C0832F99278F7099278130CD
:101860009105D9F4A9014370552702C0880F991F2B
:101870004A95E2F79C68A90164E0440F551F6A95F8
:10188000E1F744275370842B952B73E0220F331F0D
:101890007A95E1F7207633271DC08230910529F42F
:1018A000922F8827816F906A089583309105A9F45B
:1018B000A9014370552781E090E002C0880F991F6D
:1018C0004A95E2F79C6843E0220F331F4A95E1F7FF
:1018D000207E3770822B932B08950497F1F4A90191
:1018E0004370552781E090E002C0880F991F4A9508
:1018F000E2F79A68E8CFC90190578115904120F42A
:10190000C9019F7090620895C90190588115904156
:1019100020F4C9019F70906A0895203E3105E0F4DB
:10192000203C310558F52133310509F470C048F4E5
:101930002932310509F464C02A32310509F46EC038
:1019400074C029333105F1F022383105D9F025333F
:10195000310509F44EC069C0233E310589F138F4E0
:10196000203E3105C1F0223E3105E1F05EC0263E49
:10197000310569F1273E3105A9F157C0C9010E941F
:10198000CB0B08958091EA0180FD02C081FF4DC01C
:1019900080EE90E04BC08091EA0180FFF9CF89E3AF
:1019A00090E044C08091EA0182FF0EC08091EA017C
:1019B00084FF03C080E090E039C083EE90E036C041
:1019C0008091EA0182FFF2CF82EE90E02FC08091F9
:1019D000EA0183FF0BC08091EA0184FDEBCF87EE23
:1019E00090E024C08091EA0183FFF5CF86EE90E07D
:1019F0001DC08091EA0185FF07C089E290E016C012
:101A00008091EA0185FFF9CF85E390E00FC08091D6
:101A1000EA0186FF07C08AE290E008C08091EA01EF
:101A200086FFF9CF81E390E001C0C9010E94F90A65
:101A30000895089580916D0108959FB7F8941092CC
:101A40005C019FBF9091F001943009F058C09091D3
:101A5000E9009F702091EC0020FF02C020E801C047
:101A600020E0292B94E09093E9009091EB0090FF07
:101A700043C09091EE0097FF3FC090915A01992387
:101A800021F09091E80095FF37C010925A0196E03E
:101A90003091E80035FD15C03091F001343061F52A
:101AA0003091EB0035FD28C0915021F481E0809306
:101AB0005A0122C0EFE9FFE03197F1F700C00000C2
:101AC000E7CF8093F1008091E80085FD0AC0809106
:101AD000E80080FFFCCF8091E8008E778093E800DB
:101AE00006C08FB7F89491E090935C018FBF2F7080
:101AF0002093E90080E008952F702093E9008FEF94
:101B00000895CF93DF9300D01F92CDB7DEB7209119
:101B1000F001243019F523E029839B838A832093E5
:101B2000E9008FEF9091E800815095FD06C095ED9A
:101B30009A95F1F700008111F5CF8091E80085FFBB
:101B40000DC040E050E063E070E0CE0101960E94DD
:101B500050108091E8008E778093E8000F900F90EE
:101B60000F90DF91CF910895CF93DF9300D01F9214
:101B7000CDB7DEB72091F001243021F522E0298392
:101B80009B838A8383E08093E9008FEF9091E80044
:101B9000815095FD06C095ED9A95F1F700008111F1
:101BA000F5CF8091E80085FF0DC040E050E063E094
:101BB00070E0CE0101960E9450108091E8008E776F
:101BC0008093E8000F900F900F90DF91CF910895D0
:101BD0002091F0012430F1F422E02093E9002FEF6E
:101BE0003091E800215035FD06C035ED3A95F1F70A
:101BF00000002111F5CF2091E80025FF0BC040E047
:101C000050E065E070E00E9450108091E8008E770F
:101C10008093E8000895CF93DF93EC018091F00169
:101C2000843009F047C080910C018823E1F0809155
:101C30000D018823C1F085E08093E9008FEF90913A
:101C4000E800815095FD06C095E19A95F1F70000F6
:101C50008111F5CF8091E80085FF2CC040E050E075
:101C600060E170E017C081E08093E9008FEF909110
:101C7000E800815095FD06C095ED9A95F1F70000BA
:101C80008111F5CF8091E80085FF14C040E050E05D
:101C900068E070E0CE010E9450108091E8008E77DD
:101CA0008093E80080E1FE01ADE5B1E001900D9286
:101CB0008A95E1F7DF91CF91089583E993E00E943F
:101CC00052078091EF01811109C00E94E2110E9428
:101CD0003F128091E20084608093E20008958FE8D3
:101CE00093E00E9452071092EF0108958BE893E071
:101CF0000C94520787E893E00E9452070C94F42B4F
:101D000083E893E00E9452070E94CE210E94FA2BA2
:101D10000E94DB140C94190D80915B018F5F8093FE
:101D20005B0162E30E94682D911135C010925B0146
:101D300080915C01882379F18091F001843049F52C
:101D40008091E9008F709091EC0090FF02C090E8C4
:101D500001C090E0982B84E08093E9008091EB0033
:101D600080FF14C08091EE0087FF10C08091E800D2
:101D700085FF03C01092F100F9CF8091E80080FF49
:101D800005C08091E8008E778093E8009F70909363
:101D9000E90010925C01089542E061EC81E00E944C
:101DA0005C1142E061EC82E00E945C1142E061EC77
:101DB00083E00E945C1142E261EC84E00E945C11CD
:101DC00042E161EC85E00C945C118091F20183307A
:101DD00009F455C030F4813071F0823009F48EC0BE
:101DE00008958A3009F47AC08B3009F460C08930D4
:101DF00009F09CC020C08091F101813A09F096C0A1
:101E00008091E800877F8093E8008091F5019091B0
:101E1000F601892B21F060E080E090E003C060E1F2
:101E20008DE591E070E00E9499108091E8008B7739
:101E30008093E80008958091F101813209F076C025
:101E40008091F5019091F601009719F0049709F03F
:101E50006DC08091E800877F8093E8008091E80062
:101E600082FD05C08091F0018111F8CF5FC08091A3
:101E7000F10080936D018091E8008B7753C08091D1
:101E8000F101813A09F052C08091F5019091F6017B
:101E9000892B09F04BC08091E800877F8093E80090
:101EA0008091E80080FFFCCF80910C0136C08091CA
:101EB000F1018132D9F58091F5019091F601892BDC
:101EC000A9F58091E800877F8093E8000E94911136
:101ED0008091F30180930C010C94A01A8091F10180
:101EE000813221F58091E800877F8093E8000E948D
:101EF00091118091F40180936E0108958091F10118
:101F0000813AA1F48091E800877F8093E800809176
:101F1000E80080FFFCCF80916E018093F1008091FA
:101F2000E8008E778093E8000C949111089584B7AF
:101F3000877F84BF88E10FB6F89480936000109289
:101F400060000FBE90E080E80FB6F89480936100C7
:101F5000909361000FBE0E9464150E94E2110E94DE
:101F60003F128091E20084608093E2008DE19DE069
:101F70000E940D2178940E94B9140E94661582E097
:101F800091E00E94D6140E94E22B82E793E00E9427
:101F900052078091F001853089F48EE693E00E942B
:101FA00052070E9491218091EE01882391F30E94B3
:101FB000B921882371F30E943A10EBCF0E94941547
:101FC000E8CF292F332723303105A9F06CF42130D5
:101FD000310509F442C02230310509F043C08DE8D3
:101FE00090E02BEC33E042C021323105C9F02232BF
:101FF000310519F137C099278130910541F08230C0
:10200000910541F0892B71F5E7ECF3E005C0EFEAAB
:10201000F3E002C0E7E9F3E0849190E09F0126C07D
:10202000653000F5E62FF0E0EE0FFF1FEB5DFE4F91
:102030002081318189E090E019C0653098F4E62F65
:10204000F0E0DF01AA0FBB1FA55EBE4F2D913C91B2
:10205000EA5EFE4F808190E009C082E190E028E5D1
:1020600034E004C080E090E020E030E0FA01318309
:102070002083089580E189BD82E189BD09B400FE15
:10208000FDCF8091D8008F7D8093D8008091E000B3
:1020900082608093E0008091E00081FDFCCF089594
:1020A000CF92DF92EF92FF920F931F93CF93DF9324
:1020B0007C018B01EA010E94B211811131C020978D
:1020C00031F088819981081B190BE80EF91EC12C8B
:1020D000D12C0115110519F18091E80085FD14C07E
:1020E0008091E8008E778093E800209741F0888106
:1020F00099818C0D9D1D9983888385E011C00E9474
:10210000B211882331F30CC0F70181917F018093D4
:10211000F10001501109FFEFCF1ADF0ADACF80E09A
:10212000DF91CF911F910F91FF90EF90DF90CF90B3
:1021300008952091F7013091F8012617370748F0EC
:102140006115710539F42091E8002E772093E8009D
:1021500001C0B901FC0120E061157105B9F1809160
:10216000F001882309F440C0853009F43FC0809114
:10217000E80083FD3DC08091E80082FF06C08091A9
:10218000E80082FF26C080E008958091E80080FF8B
:10219000E3CF2091F3008091F20090E0922B611543
:1021A000710551F08830910538F421912093F100A8
:1021B000615071090196F3CF21E0089709F020E002
:1021C0008091E8008E778093E800C6CF2111C7CFB9
:1021D000D6CF8091F001882339F0853039F0809195
:1021E000E80083FFCCCF04C082E0089583E0089527
:1021F00081E008952091F7013091F8012617370703
:1022000048F06115710539F42091E8002E7720938C
:10221000E80001C0B901FC0120E061157105C1F1C0
:102220008091F001882309F441C0853009F440C051
:102230008091E80083FD3EC08091E80082FF06C0E7
:102240008091E80082FF27C080E008958091E80037
:1022500080FFE3CF2091F3008091F20090E0922B79
:102260006115710559F08830910540F4249120934F
:10227000F1003196615071090196F2CF21E0089783
:1022800009F020E08091E8008E778093E800C5CFC8
:102290002111C6CFD5CF8091F001882339F0853048
:1022A00039F08091E80083FFCBCF04C082E008952D
:1022B00083E0089581E00895982F973058F5909322
:1022C000E900981739F07091EC002091ED005091E1
:1022D000F00003C0242F762F50E021FF19C0309169
:1022E000EB003E7F3093EB003091ED003D7F30936B
:1022F000ED003091EB0031603093EB007093EC0017
:102300002093ED005093F0002091EE0027FF07C0CE
:102310009F5FD3CF8F708093E90081E0089580E0C4
:1023200008958091F10187FD05C08091E80080FF4C
:102330000EC012C08091E80082FD05C08091F001BE
:102340008111F8CF08958091E8008B7708C08091C3
:10235000F0018111EACF08958091E8008E77809393
:10236000E80008958091E4009091E50045E6209111
:10237000EC0020FF21C02091E80020FD21C0209129
:10238000F001222389F0253089F02091EB0025FD12
:102390000FC02091E4003091E5002817390739F388
:1023A000415041F0C901E3CF82E0089583E00895F0
:1023B00081E0089584E008952091E80022FFDFCFB6
:1023C00080E008950E9450120E945812E0EEF0E062
:1023D000808181608083E8EDF0E080818F77808369
:1023E00019BCA7EDB0E08C918E7F8C9380818F7E9D
:1023F00080831092EF0108950F931F93CF93DF9383
:102400000E9450120E945812C8EDD0E088818F7748
:10241000888388818068888388818F7D888319BCC0
:102420001092F0011092EC011092EE011092ED0169
:1024300000EE10E0F80180818B7F808388818160CD
:10244000888342E060E080E00E945C11E1EEF0E011
:1024500080818E7F8083E2EEF0E0808181608083E6
:10246000808188608083F80180818E7F808388816D
:1024700080618883DF91CF911F910F910895E8EDDE
:10248000F0E080818F7E8083E7EDF0E080818160E5
:10249000808384E082BF81E08093EF010C94FC1183
:1024A000E8EDF0E080818E7F80831092E200089555
:1024B0001092DA001092E10008951F920F920FB669
:1024C0000F9211242F933F934F935F936F937F93BA
:1024D0008F939F93AF93BF93EF93FF938091E1000E
:1024E00082FF0BC08091E20082FF07C08091E10073
:1024F0008B7F8093E1000E948C0E8091DA0080FF38
:102500001FC08091D80080FF1BC08091DA008E7FB1
:102510008093DA008091D90080FF0DC080E189BDF1
:1025200082E189BD09B400FEFDCF81E08093F00116
:102530000E945D0E05C019BC1092F0010E946F0E42
:102540008091E10080FF19C08091E20080FF15C0FA
:102550008091E2008E7F8093E2008091E2008061B2
:102560008093E2008091D80080628093D80019BCEB
:1025700085E08093F0010E947A0E8091E10084FF53
:1025800030C08091E20084FF2CC080E189BD82E1EF
:1025900089BD09B400FEFDCF8091D8008F7D809366
:1025A000D8008091E1008F7E8093E1008091E2006D
:1025B0008F7E8093E2008091E20081608093E20050
:1025C0008091EC01882311F084E007C08091E30042
:1025D00087FF02C083E001C081E08093F0010E9488
:1025E000800E8091E10083FF29C08091E20083FF8B
:1025F00025C08091E100877F8093E10082E0809395
:10260000F0011092EC018091E1008E7F8093E10057
:102610008091E2008E7F8093E2008091E2008061F1
:102620008093E20042E060E080E00E945C118091D3
:10263000F00088608093F0000E94760EFF91EF9189
:10264000BF91AF919F918F917F916F915F914F91CA
:102650003F912F910F900FBE0F901F9018951F92D2
:102660000F920FB60F9211242F933F934F935F93C6
:102670006F937F938F939F93AF93BF93CF93EF937A
:10268000FF93C091E900CF708091EC001092E900B7
:102690008091F000877F8093F00078940E946B1304
:1026A0001092E9008091F00088608093F000C09360
:1026B000E900FF91EF91CF91BF91AF919F918F91E1
:1026C0007F916F915F914F913F912F910F900FBE2E
:1026D0000F901F9018951F93CF93DF93CDB7DEB760
:1026E000AA970FB6F894DEBF0FBECDBFE1EFF1E0C1
:1026F0008091F100819321E0E93FF207C9F70E9440
:10270000E50E8091E80083FF1CC12091F10130911A
:10271000F201832F90E08A30910508F012C1FC018C
:10272000EA5AFF4F0C94882D203881F0223809F0A6
:1027300008C18091F5018F708093E9008091EB00D2
:1027400085FB882780F91092E90006C08091ED0191
:102750009091EE01911182609091E800977F9093A3
:10276000E8008093F1001092F100C5C0822F8D7FA8
:1027700009F0E7C0222319F0223061F0E2C0809115
:10278000F301813009F0DDC0333009F080E080933F
:10279000EE0128C08091F301811124C02091F50140
:1027A0002F7009F4CEC02093E9008091EB0080FFE8
:1027B00019C08091EB00333011F4806211C0806148
:1027C0008093EB0081E090E0022E01C0880F0A9414
:1027D000EAF78093EA001092EA008091EB008860AB
:1027E0008093EB001092E9008091E800877F86C01B
:1027F0002111A7C01091F3011F778091E300807829
:10280000812B8093E3008091E800877F8093E8002C
:102810000E9491118091E80080FFFCCF8091E3003D
:1028200080688093E300112311F083E001C082E00F
:102830008093F00186C02058223008F082C0809139
:10284000F3019091F4018C3D23E0920779F583E048
:102850008A838AE289834FB7F894DE01139620E0D9
:102860003EE051E2E32FF0E050935700E49120FF67
:1028700003C0E295EF703F5FEF708E2F90E0EA307B
:1028800010F0C79601C0C0968D939D932F5F2431A1
:1028900049F74FBF8091E800877F8093E8006AE2A4
:1028A00070E0CE0101960E94991014C0AE014F5FF6
:1028B0005F4F6091F5010E94E10F009709F441C05C
:1028C0002091E800277F2093E800BC0189819A814C
:1028D0000E94FA108091E8008B778093E80031C065
:1028E000203879F58091E800877F8093E800809117
:1028F000EC018093F1008091E8008E778093E800EE
:102900000E9491111EC021111CC09091F3019230C0
:10291000C0F48091E800877F8093E8009093EC01F9
:102920000E9491118091EC01811104C08091E3001B
:1029300087FF02C084E001C081E08093F0010E9423
:10294000CC0E8091E80083FF0AC08091E800877F69
:102950008093E8008091EB0080628093EB00AA9660
:102960000FB6F894DEBF0FBECDBFDF91CF911F91A0
:102970000895CF938091F0018823B1F08091E90010
:102980008F709091EC0090FF02C090E801C090E041
:10299000C92FC82B1092E9008091E80083FD0E94A6
:1029A0006B13CF70C093E900CF9108959093740199
:1029B000809373010895E0917301F0917401309751
:1029C00021F00190F081E02D099480E00895FF92BC
:1029D0000F931F93CF93DF938C01E0917301F091DC
:1029E0007401309799F10280F381E02D099580916F
:1029F000D70182FF2BC080FF04C08DE895E00E94C4
:102A00005207E80180E1F82E07E815E08091D70130
:102A100080FF0BC088811F928F931F930F930E949A
:102A2000EB070F900F900F900F90FA942196F110F2
:102A3000EDCF8091D70180FF09C085E895E0DF9157
:102A4000CF911F910F91FF900C945207DF91CF917E
:102A50001F910F91FF900895E0917301F09174011F
:102A6000309721F00480F581E02D0994089520919C
:102A70007101309172018217930771F09093720186
:102A800080937101E0917301F0917401309721F00E
:102A90000680F781E02D0994089520916F0130910F
:102AA00070018217930771F09093700180936F010A
:102AB000E0917301F0917401309721F00084F18569
:102AC000E02D0994089508950C9463150E94D02177
:102AD0000E9464090C949622CF93C82F8091D7014D
:102AE00082FF1EC080FF04C086EA95E00E94520764
:102AF0008091D70180FF0CC01F92CF9321EA35E06F
:102B00003F932F930E94EB070F900F900F900F9021
:102B10008091D70180FF04C08FE995E00E945207A1
:102B20008C2FCF910C94190DCF92DF92EF92FF92E0
:102B30000F931F93CF93DF93CDB7DEB72B970FB6CD
:102B4000F894DEBF0FBECDBF0E94810936E7E32EA9
:102B500031E0F32E00E010E0C02E802F0E94AC0A7E
:102B6000F701D1907F01D826B1F40F5F1F4F0E30CF
:102B7000110591F78FEF89838A831B820E94D921E7
:102B80008160782F9D838C8349815A816B818D81EF
:102B90000E94371641C09091D70191FF04C08B87E6
:102BA0000E94B20A8B8520E030E04D2D50E0922F3C
:102BB000BA01022E02C0759567950A94E2F760FF8C
:102BC00025C02E83CF82EE24E394F12C02C0EE0CBC
:102BD000FF1C9A95E2F790E08E219F2121E0892B3E
:102BE00009F420E028870E94D9218160782F9A87F4
:102BF00089874E815F8168858A850E943716F80132
:102C0000EA58FE4F80818E25808306C02F5F3F4F9C
:102C10002630310561F6A9CF0E9404261091750176
:102C20000E94DB141817A1F00E94DB148093750139
:102C30002B960FB6F894DEBF0FBECDBFDF91CF91BC
:102C40001F910F91FF90EF90DF90CF900C946C1537
:102C50002B960FB6F894DEBF0FBECDBFDF91CF919C
:102C60001F910F91FF90EF90DF90CF900895CF9339
:102C7000DF93CDB7DEB72B970FB6F894DEBF0FBE4C
:102C8000CDBF4F83588769877A878B87DE0111967E
:102C900086E0FD0111928A95E9F785E0FE013796FD
:102CA00001900D928A95E1F749815A816B817C816F
:102CB0008D819E810E946C1D2B960FB6F894DEBF0D
:102CC0000FBECDBFDF91CF910895CF93C82F88233A
:102CD00009F4C1C0823859F40E94DB1481FDBBC0E5
:102CE00089E30E940B200E94E72089E30CC083380F
:102CF00079F40E94DB1480FDAEC083E50E940B20B6
:102D00000E94E72083E50E945C20CF910C94E7208D
:102D1000843859F40E94DB1482FD9DC087E40E9430
:102D20000B200E94E72087E4EECF8CEF8C0F813AD6
:102D300048F48C2F0E948D2A81118DC08C2F0E9407
:102D40000B20E3CF80E28C0F883048F4C77081E01D
:102D500001C0880FCA95EAF70E94AE20D6CF8BE556
:102D60008C0F833078F4C53A29F0C63A31F482E802
:102D700090E005C081E890E002C083E890E0CF9148
:102D80000C94371588E58C0F833108F064C0C83A7D
:102D900039F1C93A41F1CA3A49F1CB3A51F1CC3A49
:102DA00059F1CD3A61F1C03B69F1CE3A71F1CF3AB8
:102DB00079F1C13B81F1C23B89F1C33B91F1C43B45
:102DC00099F1C53BA1F1C63BA9F1C73BB1F1C83BA5
:102DD000B9F1C93BC1F1CA3BC9F58AE292E038C0FA
:102DE00082EE90E035C089EE90E032C08AEE90E04D
:102DF0002FC085EB90E02CC086EB90E029C087EBDC
:102E000090E026C08CEC90E023C08DEC90E020C0D8
:102E100083E891E01DC08AE891E01AC082E991E060
:102E200017C084E991E014C081E292E011C083E20E
:102E300092E00EC084E292E00BC085E292E008C00E
:102E400086E292E005C087E292E002C080E090E076
:102E5000CF910C944D15CF910895882309F44BC060
:102E6000823859F40E94DB1481FF45C089E30E9437
:102E70000B200E94E72089E30CC0833871F40E9484
:102E8000DB1480FF38C083E50E940B200E94E720FE
:102E900083E50E945C200C94E720843859F40E945A
:102EA000DB1482FF28C087E40E940B200E94E720E9
:102EB00087E4EFCF9CEF980F913A58F390E2980F88
:102EC000983050F4877091E001C0990F8A95EAF725
:102ED000892F0E94B420DFCF9BE5980F933020F418
:102EE00080E090E00C943715885A833120F480E01C
:102EF00090E00C944D150895882321F00E94AE2097
:102F00000C94E7200895882321F00E94B4200C94AB
:102F1000E7200895CF92DF92EF92FF920F931F93D5
:102F2000CF93DF93CDB7DEB728970FB6F894DEBF07
:102F30000FBECDBF8C0185E0F801DE011196019036
:102F40000D928A95E1F7F80140813181F280258167
:102F500022952F7083819481892B31F03F3F31F48A
:102F600081E04F3F19F403C081E001C080E080FDA3
:102F7000C6C249833A8389819A812F830E94C91FDF
:102F80009E8388870E94C81F0E949B1E4E81E42F4B
:102F9000E295EF70F0E0E05AFF4F2F8168850C94C6
:102FA000882D842F807F142F1F70882311F0129595
:102FB000107FFF2059F0112309F456C2812F688732
:102FC0000E94BE200E94E72068854EC2862F0E9484
:102FD0002D17112309F493C2812F0E94C420289633
:102FE0000FB6F894DEBF0FBECDBFDF91CF911F911A
:102FF0000F91FF90EF90DF90CF900C94E720342F4B
:10300000307F842F8F70303211F08295807F66235D
:1030100019F0613019F12CC0FF20B1F0222309F41E
:1030200094C1213009F091C128960FB6F894DEBF03
:103030000FBECDBFDF91CF911F910F91FF90EF9009
:10304000DF90CF900C94CE20222319F0213009F488
:1030500056C28E830E94D1208E818AC1FF2021F02A
:10306000263008F04CC271C1253008F048C280C13A
:10307000FF2021F0222309F468C1F6C1222309F4BC
:1030800077C106C2242F26952695237030E021159E
:10309000310521F021303105C9F031C2FF2021F086
:1030A000862F942F937002C080E090E028960FB690
:1030B000F894DEBF0FBECDBFDF91CF911F910F916E
:1030C000FF90EF90DF90CF900C943715FF2021F008
:1030D000862F942F937002C080E090E028960FB660
:1030E000F894DEBF0FBECDBFDF91CF911F910F913E
:1030F000FF90EF90DF90CF900C944D15862FFF201E
:1031000019F00E948A2402C00E94F22428960FB669
:10311000F894DEBF0FBECDBFDF91CF911F910F910D
:10312000FF90EF90DF90CF900C947725842F8370E1
:1031300009F076C0F110E3C1262F2295269527705D
:10314000220F220F862F8F70C82ED12CE12CF12C4C
:10315000022E04C0CC0CDD1CEE1CFF1C0A94D2F71E
:1031600064FF10C06FE070E080E090E004C0660F84
:10317000771F881F991F2A95D2F7609570958095C3
:10318000909503C060E070E0CB01242F2695269532
:103190002370422F50E042305105D1F043305105A9
:1031A00059F16C297D298E299F294130510541F122
:1031B00028960FB6F894DEBF0FBECDBFDF91CF913A
:1031C0001F910F91FF90EF90DF90CF900C94C01E55
:1031D0006C297D298E299F2928960FB6F894DEBF89
:1031E0000FBECDBFDF91CF911F910F91FF90EF9058
:1031F000DF90CF900C94DA1E0E94C01EC701B6016A
:1032000028960FB6F894DEBF0FBECDBFDF91CF91E9
:103210001F910F91FF90EF90DF90CF900C94A61E1E
:10322000FF2019F0842F817001C08695882309F44E
:1032300066C1262F229526952770220F220F862FF2
:103240008F70C82ED12CE12CF12C022E04C0CC0C96
:10325000DD1CEE1CFF1C0A94D2F764FF10C06FE067
:1032600070E080E090E004C0660F771F881F991F10
:103270002A95D2F7609570958095909503C060E08F
:1032800070E0CB01242F269526952370422F50E025
:1032900042305105D1F04330510559F16C297D2957
:1032A0008E299F294130510541F128960FB6F89497
:1032B000DEBF0FBECDBFDF91CF911F910F91FF9069
:1032C000EF90DF90CF900C94941F6C297D298E296C
:1032D0009F2928960FB6F894DEBF0FBECDBFDF91B1
:1032E000CF911F910F91FF90EF90DF90CF900C94B2
:1032F000AE1F0E94941FC701B60128960FB6F8941E
:10330000DEBF0FBECDBFDF91CF911F910F91FF9018
:10331000EF90DF90CF900C947A1F603FC9F118F4C2
:10332000603E50F49CC0623F09F461C008F44BC099
:10333000633F09F470C093C0162F1F70842F8F71E4
:10334000FF2099F00E94131F812F28960FB6F89442
:10335000DEBF0FBECDBFDF91CF911F910F91FF90C8
:10336000EF90DF90CF900C947C170E94341F812F38
:1033700028960FB6F894DEBF0FBECDBFDF91CF9178
:103380001F910F91FF90EF90DF90CF900C948317D7
:10339000FF20A9F0253008F0B2C0842F8F71289645
:1033A0000FB6F894DEBF0FBECDBFDF91CF911F9156
:1033B0000F91FF90EF90DF90CF900C94591F263023
:1033C00008F09DC0EACFFF20A1F0842F8F712896CE
:1033D0000FB6F894DEBF0FBECDBFDF91CF911F9126
:1033E0000F91FF90EF90DF90CF900C94131FFF2070
:1033F00061F3842F8F7128960FB6F894DEBF0FBE4D
:10340000CDBFDF91CF911F910F91FF90EF90DF9093
:10341000CF900C94341FFF2091F0842F8F71289649
:103420000FB6F894DEBF0FBECDBFDF91CF911F91D5
:103430000F91FF90EF90DF90CF900C94FE1E289696
:103440000FB6F894DEBF0FBECDBFDF91CF911F91B5
:103450000F91FF90EF90DF90CF900C94F41EFF201F
:10346000A1F0222309F4B1CF862F28960FB6F89445
:10347000DEBF0FBECDBFDF91CF911F910F91FF90A7
:10348000EF90DF90CF900C946516222309F4B1CF12
:10349000862F28960FB6F894DEBF0FBECDBFDF9102
:1034A000CF911F910F91FF90EF90DF90CF900C94F0
:1034B0002D174F70C8010E94F40728960FB6F89494
:1034C000DEBF0FBECDBFDF91CF911F910F91FF9057
:1034D000EF90DF90CF900C94191E4F70C801289682
:1034E0000FB6F894DEBF0FBECDBFDF91CF911F9115
:1034F0000F91FF90EF90DF90CF900C94B80B28962F
:103500000FB6F894DEBF0FBECDBFDF91CF911F91F4
:103510000F91FF90EF90DF90CF9008950E94CB2005
:103520000E94A0200E94E7200E94A5260E947725E5
:1035300080E090E00E94371580E090E00C944D15FB
:103540000E94BB200C948E1A0E94C91F292F22951D
:103550002F7030E02C3031054CF42A3031056CF4FA
:10356000225031092230310590F407C02C3031054A
:1035700051F02F30310539F00AC0803E10F0803F05
:1035800031F481E0089593FB882780F9089580E065
:103590000895CF93DF9300D000D01F92CDB7DEB750
:1035A0000F900F900F900F900F90DF91CF91089593
:1035B000CF93DF9300D000D000D0CDB7DEB72696F2
:1035C0000FB6F894DEBF0FBECDBFDF91CF91089547
:1035D0001F93CF93DF93C091840116E08091850102
:1035E000C81799F0D0E01C9FF0011D9FF00D112429
:1035F000EA57FE4F408151816281738184819581B8
:103600000E94D81A2196C770E9CFDF91CF911F9100
:1036100008954091B6015091B7016091B801709141
:10362000B9018091BA019091BB010C94D81ACF9343
:103630008091BB0182958F7009F05FC08091B801C5
:10364000882309F45AC020918401A09185016091DA
:10365000B6017091B7018091B9019091BA0131E042
:103660006F3F09F030E0B32FC6E02A1709F445C0D8
:10367000009721F07F3F21F44B2F03C041E001C0B0
:1036800040E030E040FD35C0C29FF001C39FF00D27
:103690001124EA57FE4F418174132BC040816413FB
:1036A00028C04281411125C04381548148175907E0
:1036B00010F441505109481B590B483C5105C8F4BE
:1036C0008091BB018F7080618093BB0186E0829FF7
:1036D000F001839FF00D1124E557FE4F80818F701C
:1036E0008061808386EB91E00E948A17CF910C94D1
:1036F000E81A2F5F3F4F2770B8CFCF910895CF9230
:10370000DF92EF92FF920F931F93CF93DF93CDB78A
:10371000DEB762970FB6F894DEBF0FBECDBF8C0147
:1037200085E0F801DE011D9601900D928A95E1F782
:10373000D8014C9111965C91119712966C91129749
:103740001396ED90FC9014977091B601E091B7013B
:103750002091B9013091BA012115310531F0EF3FC7
:1037600031F481E07F3F19F403C081E001C080E0C3
:10377000B82FB170CB2E80FD6CC1D090B801DD2088
:1037800009F4F5C0F091BB01E216F30638F0C70169
:10379000821B930B883C910548F09BC02095309587
:1037A0002E0D3F1D283C310508F093C08F2F807FE0
:1037B00009F052C0E51314C0741312C0D62E611163
:1037C0000FC0FF70F061F093BB010E94091B86EBF4
:1037D00091E00E948A178091BB01F80185836CC13A
:1037E000EF2831F05F3F31F481E04F3F19F403C01F
:1037F00081E001C080E080FD03C081E0862701C038
:1038000080E0F82FF170FF2E80FF1CC080918401B2
:103810002091850136E0821709F428C190E0389F95
:10382000F001399FF00D1124EA57FE4F71815713B3
:1038300006C07081471303C07281671303C00196ED
:103840008770E9CFD62E662309F436C18091BB017B
:1038500081608093BB0153C0E51308C0741306C098
:10386000611104C0D8011596FC93AEC04D875E87E8
:103870008D859E856A8B0E94A41A6A89882329F106
:10388000D62E662311F12091BB01822F82958F7075
:1038900090E002970CF460C08091B6019091B7015E
:1038A00098878F831986FB86EA862C87CE01079638
:1038B00051C0E51731F14D875E878D859E856A8BF6
:1038C0000E94A41A6A8981112EC0C8010E948A1719
:1038D000A4C08F2F807F69F77E2DF98AE88A8989B5
:1038E0000E94C91A86EB91E00E948A17E6EBF1E08C
:1038F00086E0DF011D928A95E9F70E94091BD12C11
:10390000DBC07413D8CF6111D6CFD8011596FC93C4
:10391000C8010E948A17E6EBF1E086E0DF011D9204
:103920008A95E9F7C9C0D62E662379F22091BB01AA
:10393000822F82958F7090E0029774F08091B6018B
:103940009091B7019A8389831B82FD82EC822E833A
:10395000CE0101960E948A1786E0F801A6EBB1E03D
:1039600001900D928A95E1F70E94171B6FC0E21635
:10397000F30628F0C701821B930B9C0104C020951D
:1039800030952E0D3F1D283C310508F052C0D62E33
:10399000662309F49ACFE5132CC074132AC08091D2
:1039A000BB0180FD1DC0982F92959F70C9F0D80172
:1039B00015968C9315979F3039F09F5F9295907F65
:1039C0008F70892B15968C93C8010E948A1786E008
:1039D000F801A6EBB1E001900D928A95E1F736C0AF
:1039E00086E0F801A6EBB1E001900D928A95E1F72F
:1039F00063C04D875E878D859E850E94A41A8823AB
:103A000079F086E0F801A6EBB1E001900D928A957D
:103A1000E1F70E94171B0E94091BDD24D3944CC0C0
:103A20008091BB0181608093BB01C8010E948A170D
:103A300043C07E2DF98AE88A89890E94C91AE6EB7B
:103A4000F1E086E0DF011D928A95E9F70E94091BEB
:103A500033C0662309F439CF4D875E878D859E85F7
:103A60000E94A41A882309F430CFCBCF4D875E87FC
:103A70008D859E850E94C91F292F22952F7030E0C9
:103A8000223031052CF49F7041F0811106C00CC02A
:103A9000243031052CF49F7049F4805E883020F08A
:103AA000C8010E948A17CF2CDC2C06C0D8011596BD
:103AB0009C91907F91F7F8CF8D2D62960FB6F89478
:103AC000DEBF0FBECDBFDF91CF911F910F91FF9051
:103AD000EF90DF90CF9008951F93CF93DF93CDB7F2
:103AE000DEB72C970FB6F894DEBF0FBECDBF4F8365
:103AF000588769877A878B879C87CE0107960E94B3
:103B00007F1B8823C1F02F8138858A859B85892B6F
:103B100031F03F3F11F080E003C02F3FE1F781E03B
:103B2000811147C04F81588569857A858B859C8531
:103B30000E94D81A3EC086E0FE013796DE0111963B
:103B400001900D928A95E1F7FF81E8854A855B85B2
:103B50004115510531F0EF3F31F481E0FF3F19F499
:103B600003C081E001C080E080FD23C02091850179
:103B700030E0C9010196877099276091840170E057
:103B800086179707F1F1F983EA835D834C8396E00A
:103B9000929FD001939FB00D1124AA57BE4FFE01F2
:103BA000319601900D929A95E1F7809385010E94DC
:103BB000E81A16E08091840190918501891779F1C6
:103BC000189FC00111248A579E4F0E947F1B882393
:103BD00031F1E09184011E9FF0011124EA57FE4F5C
:103BE0004081518162817381848195810E94D81ABC
:103BF0008091840190E001968770992780938401D9
:103C0000D9CF0E94A01A1092850110928401E6EB90
:103C1000F1E086E0DF011D928A95E9F7CACF2C9684
:103C20000FB6F894DEBF0FBECDBFDF91CF911F91CD
:103C30000895EF92FF920F931F93CF93DF939C0110
:103C4000009709F471C0F12CEE24E394E901219668
:103C5000F9018491843740F4843008F056C08130F3
:103C600081F0823021F160C0853709F449C0C0F18C
:103C70009CE7980F903708F057C08F770E942D1758
:103C800046C089010E5F1F4FFE01849190E2980F9C
:103C9000983050F48770FE2D01C0FF0F8A95EAF727
:103CA0008F2F0E94BE2015C00E94651614C0890186
:103CB0000E5F1F4FFE01849190E2980F983068F4D8
:103CC0008770FE2D01C0FF0F8A95EAF78F2F0E94A3
:103CD000C4200E94E720E8011AC00E942D17FBCFE4
:103CE0002E5F3F4FFE01C491CC2341F08FE99FE04E
:103CF0000197F1F700C00000C150F6CFE90107C0FD
:103D0000FE01F490E901229602C00E9465168F2DF3
:103D1000882341F0EFE9FFE03197F1F700C00000A0
:103D20008150F6CF9E0192CFDF91CF911F910F91DD
:103D3000FF90EF90089508956093C0017093C101C2
:103D40008093C2019093C3010C948E1A0F931F931A
:103D50000091C0011091C1012091C2013091C301B5
:103D6000062B172B282B392B0093C0011093C10170
:103D70002093C2013093C3011F910F910C948E1AAE
:103D80000F931F930091C0011091C1012091C201B6
:103D90003091C30106231723282339230093C00140
:103DA0001093C1012093C2013093C3011F910F9161
:103DB0000C948E1A0F931F930091C0011091C101B2
:103DC0002091C2013091C3010627172728273927E0
:103DD0000093C0011093C1012093C2013093C3012D
:103DE0001F910F910C948E1A1092BC011092BD017C
:103DF0001092BE011092BF010C948E1A41E050E067
:103E000060E070E004C0440F551F661F771F8A955D
:103E1000D2F74093BC015093BD016093BE017093F3
:103E2000BF010C948E1A41E050E060E070E004C0E5
:103E3000440F551F661F771F8A95D2F78091BC01EA
:103E40009091BD01A091BE01B091BF01842B952B33
:103E5000A62BB72B8093BC019093BD01A093BE010C
:103E6000B093BF010C948E1A41E050E060E070E026
:103E700004C0440F551F661F771F8A95D2F74095DF
:103E80005095609570958091BC019091BD01A09175
:103E9000BE01B091BF0184239523A623B72380934D
:103EA000BC019093BD01A093BE01B093BF010C94DF
:103EB0008E1A41E050E060E070E004C0440F551FEE
:103EC000661F771F8A95D2F78091BC019091BD0142
:103ED000A091BE01B091BF0184279527A627B727DF
:103EE0008093BC019093BD01A093BE01B093BF012C
:103EF0000C948E1A0F931F930091BC011091BD0179
:103F00002091BE013091BF01062B172B282B392B96
:103F10000093BC011093BD012093BE013093BF01FB
:103F20001F910F910C948E1A0F931F930091BC0157
:103F30001091BD012091BE013091BF0106231723CE
:103F4000282339230093BC011093BD012093BE01A7
:103F50003093BF011F910F910C948E1A0F931F93F2
:103F60000091BC011091BD012091BE013091BF01B3
:103F700006271727282739270093BC011093BD0176
:103F80002093BE013093BF011F910F910C948E1AA4
:103F90000895CF92DF92EF92FF920F931F93CF93EA
:103FA000DF93EC01C090C001D090C101E090C2014C
:103FB000F090C3018091BC019091BD01A091BE0120
:103FC000B091BF01C82AD92AEA2AFB2A0FE110E0E2
:103FD000B701A601002E04C07695679557954795C1
:103FE0000A94D2F740FF07C0BE01802F0E94DB0B6E
:103FF0008130910539F40150110950F7BE0180E07C
:104000000E94DB0BDF91CF911F910F91FF90EF90FA
:10401000DF90CF90089590910C01992361F19091D8
:104020000D01992341F1982F9695969596959F307D
:1040300088F4E0910E01F0910F01E90FF11D8770F6
:1040400021E030E001C0220F8A95EAF78181822BBE
:10405000818308959091D70190FF2DC01F928F9377
:1040600087ED95E09F938F930E94EB070F900F9041
:104070000F900F90089540910E0150910F0120E094
:1040800030E09FEFFA01E20FF31F6281681799F0A9
:104090009F3F19F4611101C0922F2F5F3F4F2E30C7
:1040A000310581F79F3F39F0FA01E90FF11D97FDC6
:1040B000FA9582830895089590910C01992369F1EE
:1040C00090910D01992349F1982F96959695969583
:1040D0009F3090F4E0910E01F0910F01E90FF11D76
:1040E000877021E030E001C0220F8A95EAF7209521
:1040F00081812823218308959091D70190FF1FC0CB
:104100001F928F9389EB95E09F938F930E94EB070B
:104110000F900F900F900F90089540910E015091C5
:104120000F0120E030E0FA01E20FF31F92819813B3
:1041300001C012822F5F3F4F2E303105A1F7089545
:1041400081E090E0E0910E01F0910F01E80FF91F7E
:104150001082019680319105A9F708959091D601BA
:10416000982B9093D601089580959091D60198232D
:104170009093D60108951092D60108959091D5019B
:10418000982B9093D501089580959091D50198230F
:104190009093D50108951092D50108958093C4019C
:1041A00008951092C401089540910E0150910F019D
:1041B00020E030E080E0FA01E20FF31F91819111DD
:1041C0008F5F2F5F3F4F2F303105A9F70895E091A2
:1041D0000E01F0910F018091D6018083E0910E01D4
:1041E000F0910F0180819091D501892B808390916E
:1041F000C401992361F0E0910E01F0910F018081DB
:10420000892B80830E94D42081111092C401809157
:104210000E0190910F010C94E71490933B01809351
:104220003A010895CF92DF92EF92FF920F931F937E
:104230006C01EE24FF24C114D104E104F10421F443
:104240006B017C0180E001C080E133272F2D1E2D02
:104250000D2D011511052105310519F0885F680143
:10426000790197018601A4E0369527951795079562
:10427000AA95D1F7011511052105310519F08C5FBB
:104280006801790197018601F2E036952795179527
:104290000795FA95D1F7011511052105310519F09A
:1042A0008E5F68017901B701A601769567955795EC
:1042B0004795452B462B472B09F08F5F1F910F9198
:1042C000FF90EF90DF90CF9008958295982F9C7C7F
:1042D00096959695837344E0849F90011124922BC8
:1042E000892F8A7A86959575990F892B08951F9342
:1042F000CF93DF931F92CDB7DEB799830E946521DC
:10430000182F9981892F0E946521212F30E0322FAB
:104310002227A901482BCA010F90DF91CF911F914D
:1043200008958091F001843009F11092D80120E4C1
:1043300088E190E00FB6F894A895809360000FBED6
:104340002093600083B7817F846083BF83B78160DF
:1043500083BF7894889583B78E7F83BF88E10FB63B
:10436000F89480936000109260000FBE0895089545
:104370000895CF930E94B7210E9481090E94B8211D
:10438000C0E08C2F0E94AC0A811105C0CF5FCE30F7
:10439000C1F780E001C081E0CF9108950C94A01A8C
:1043A00082E084BD93E095BD9AEF97BD80936E0047
:1043B00008952FB7F8948091D9019091DA01A091D6
:1043C000DB01B091DC012FBF0895CF92DF92EF9215
:1043D000FF920F931F932FB7F8944091D9015091FA
:1043E000DA016091DB017091DC012FBF6A017B0172
:1043F000EE24FF248C0120E030E0C016D106E20656
:10440000F30610F441505109481B590BCA011F9182
:104410000F91FF90EF90DF90CF9008951F920F9231
:104420000FB60F9211248F939F93AF93BF938091F8
:10443000D9019091DA01A091DB01B091DC010196E4
:10444000A11DB11D8093D9019093DA01A093DB01E6
:10445000B093DC01BF91AF919F918F910F900FBEF0
:104460000F901F9018950E94E211F8942FEF87EAA1
:1044700091E6215080409040E1F700C0000087E0C5
:1044800090EBDC018093F9019093FA01A093FB017A
:10449000B093FC012CE088E190E00FB6F894A89569
:1044A000809360000FBE20936000FFCFEF92FF92D9
:1044B0000F931F93CF93DF93E82EF12C8F2D0E9443
:1044C000AC0AC0E0D0E0082F10E098010C2E02C02A
:1044D000359527950A94E2F720FD05C02196C63050
:1044E000D10599F709C06C2F7F2D80E00E94B90B90
:1044F000E812F4CF81E005C0F3948EE0F812DECF2D
:1045000080E0DF91CF911F910F91FF90EF90089580
:10451000CF93C82F8CE20E945622882321F08C2F43
:10452000CF910C94562280E0CF910895CF930E94B2
:10453000E323811102C00E94C9238CEF95E00E9401
:104540005207C5E6C15049F00E9481098FE39CE9FA
:104550000197F1F700C00000F5CF85EF95E00E94CC
:10456000520789E20E948822811111C18AE20E94C9
:10457000882281110E94C92385E00E94882281112E
:104580000E9433220E94EE238093D70187E00E948D
:104590008822882399F18BE10E948822882351F098
:1045A0009091D70191FB882780F921E0822780FB39
:1045B00091F922C08EE00E948822882351F09091C8
:1045C000D70192FB882780F921E0822780FB92F9AE
:1045D00013C080E10E9488229091D701882341F086
:1045E00093FB882780F921E0822780FB93F904C0A0
:1045F000892F809580FB90F99093D7018091D70106
:104600000E94F2230E9400248093EA0180EE0E941F
:104610008822882341F08091EA01982F909590FBA1
:1046200080F98093EA0189E30E948822882359F067
:104630009091EA0191FB882780F921E0822780FB95
:1046400091F99093EA0182EE0E948822882359F022
:104650009091EA0192FB882780F921E0822780FB74
:1046600092F99093EA0186EE0E948822882359F0FD
:104670009091EA0193FB882780F921E0822780FB53
:1046800093F99093EA0183EE0E948822882359F0DF
:104690009091EA0194FB882780F921E0822780FB32
:1046A00094F99093EA0185E30E948822882359F0C7
:1046B0009091EA0195FB882780F921E0822780FB11
:1046C00095F99093EA0181E30E948822882359F0AA
:1046D0009091EA0196FB882780F921E0822780FBF0
:1046E00096F99093EA0181E10E948822882359F08B
:1046F0009091EA0197FB882780F921E0822780FBCF
:1047000097F99093EA018091EA010E940424809134
:10471000EA0187FB882780F980930D0187E20E94D8
:104720008822C82F8EE10E9488228111C2608FE109
:104730000E9488228111C46080E20E948822811137
:10474000C86081E20E9488228111C06182E20E94D9
:1047500088228111C06283E20E9488228111C06494
:1047600084E20E948822882311F0C06802C0CC2312
:1047700029F08C2F0E94FB236C2F03C00E94F7238B
:10478000682F70E080E090E0CF910C949C1ECF9158
:1047900008956DEE7EEF80E090E00E94BE2D60E017
:1047A00082E090E00E94B02D60E083E090E00E9403
:1047B000B02D60E084E090E00E94B02D60E085E0E4
:1047C00090E00C94B02D80E090E00E94AA2D21E0B2
:1047D0008D3E9E4F09F020E0822F089582E090E008
:1047E0000C94A22D682F82E090E00C94B02D83E011
:1047F00090E00C94A22D682F83E090E00C94B02DF3
:1048000084E090E00C94A22D682F84E090E00C945A
:10481000B02D8091DF0180FF0BC06091130185E016
:10482000689FB001112475956795759567952AC0A5
:1048300081FF09C06091130185E0689FB0011124D8
:10484000759567951FC082FF07C06091130185E0D1
:10485000689FB001112416C04091E0014423C9F0C3
:1048600060911201461788F72091130185E0289F77
:1048700090011124429FC001439F900D112470E0CC
:104880000E94742D6038710540F46115710539F08E
:1048900002C065E070E0862F08958FE7089581E0FB
:1048A00008958091DF0180FF08C06091110170E0E0
:1048B000759567957595679521C081FF06C06091D4
:1048C000110170E07595679519C082FF04C0609171
:1048D000110170E010C08091E0018823C1F0609167
:1048E00010018617A0F790911101989FC001112423
:1048F00070E00E94742D6038710528F4611571050F
:1049000021F0862F08958FE7089581E0089561E0F2
:1049100070E0F4CF803F21F40E940924819504C007
:10492000813F29F40E9409248093E3010895823F86
:1049300021F40E940924819504C0833F29F40E9438
:1049400009248093E2010895893F19F40E945124BB
:1049500005C08A3F31F40E94512481958093E4017F
:1049600008958B3F21F40E945124819504C08C3F0F
:1049700029F40E9451248093E5010895843F21F495
:104980008091E101816017C0853F21F48091E101B0
:10499000826011C0863F21F48091E10184600BC0E8
:1049A000873F21F48091E101886005C0883F31F4A0
:1049B0008091E10180618093E10108958D3F21F4B0
:1049C0008091DF0181600BC08E3F21F48091DF0177
:1049D000826005C08F3F29F48091DF01846080935D
:1049E000DF010895803F39F48091E30187FF6CC0B7
:1049F0001092E30169C0813F29F48091E301181608
:104A0000BCF362C09091E201823F29F497FF5CC041
:104A10001092E20159C0833F19F41916CCF354C027
:104A2000893F41F48091E40118160CF04DC01092BA
:104A3000E4014AC08A3F29F48091E40187FF44C021
:104A4000F6CF8B3F39F48091E50187FF3DC010928E
:104A5000E5013AC08C3F29F48091E5011816BCF3BA
:104A600033C0843F21F48091E1018E7F17C0853FE0
:104A700021F48091E1018D7F11C0863F21F4809166
:104A8000E1018B7F0BC0873F21F48091E101877F9B
:104A900005C0883F31F48091E1018F7E8093E10170
:104AA00013C08D3F21F48091DF018E7F0BC08E3FBC
:104AB00021F48091DF018D7F05C08F3F29F4809123
:104AC000DF018B7F8093DF018091E20181110EC0B5
:104AD0008091E30181110AC08091E401811106C037
:104AE0008091E501811102C01092E001089580914A
:104AF000D70183FF7EC088E396E00E945207809131
:104B0000E1011F928F9383E396E09F938F930E941E
:104B1000EB0781E396E00E9452072091E201822F89
:104B2000992787FD90959F932F938EE296E09F9310
:104B30008F930E94EB078CE296E00E94520720912F
:104B4000E301822F992787FD90959F932F9389E208
:104B500096E09F938F930E94EB0787E296E00E9476
:104B600052072091E401822F992787FD90959F930A
:104B70002F9384E296E09F938F930E94EB0782E24B
:104B800096E00E9452072091E501822F992787FD28
:104B900090959F932F938FE196E09F938F930E9420
:104BA000EB078CE196E00E9452078091E0011F9292
:104BB0008F9389E196E09F938F930E94EB0787E1A3
:104BC00096E00E9452078091DF011F928F9384E14B
:104BD00096E09F938F930E94EB0781E196E00E94FD
:104BE00052078DB79EB74C960FB6F8949EBF0FBE76
:104BF0008DBF81EE91E00E942C150E94D9219093E7
:104C0000DE018093DD0108951F93CF93DF938091A0
:104C1000DD019091DE010E94E5214091E0014423F5
:104C200021F02091140130E006C0209115015AE0D6
:104C3000259F900111248217930708F482C0809168
:104C4000E2011091E301D091E401C091E5018111ED
:104C500007C0111105C0D11103C0CC2309F471C0E4
:104C60004F3F19F04F5F4093E001181624F40E9463
:104C700009248093E2018091E20187FF05C00E9430
:104C8000092481958093E201111624F40E940924DD
:104C90008093E3018091E30187FF05C00E9409240E
:104CA00081958093E3016091E201662339F11091CF
:104CB000E301112319F1772767FD7095872F972F4F
:104CC0000E94792C23E333E343E35FE30E94DD2C6E
:104CD0000E94462C6093E201612F772767FD709553
:104CE000872F972F0E94792C23E333E343E35FE37D
:104CF0000E94DD2C0E94462C6093E3011D1624F4D3
:104D00000E9451248093E4018091E40187FF05C053
:104D10000E94512481958093E4011C1624F40E9482
:104D200051248093E5018091E50187FF05C00E9431
:104D3000512481958093E501DF91CF911F910C94CF
:104D40007725DF91CF911F910895E1EEF1E085E0A5
:104D5000DF011D928A95E9F71092E0011092DF01C0
:104D600008958BE598E00E9452071F9281E08F938F
:104D70001F9285E08F938DE098E09F938F930E9420
:104D8000EB070F900F900F900F900F900F900895DA
:104D90008330E9F128F4813061F0823009F108951F
:104DA000853009F462C008F449C0863009F474C043
:104DB000089520911501862F90E0820F911D8F3F5D
:104DC000910520F4620F6093150103C08FEF80936B
:104DD0001501809115011F928F9386E497E072C0B0
:104DE00020911401862F90E0820F911D8F3F910535
:104DF00020F4620F6093140103C08FEF80931401BD
:104E0000809114011F928F9384E397E05BC02091FF
:104E10001301862F90E0820F911D8F3F910520F4A2
:104E2000620F6093130103C08FEF80931301809191
:104E300013011F928F9381E297E044C020911201E9
:104E4000862F90E0820F911D8F3F910520F4620F15
:104E50006093120103C08FEF8093120180911201C1
:104E60001F928F938CE097E02DC020911101862F27
:104E700090E0820F911D8F3F910520F4620F6093A7
:104E8000110103C08FEF80931101809111011F92D6
:104E90008F9383EF96E016C020911001862F90E04B
:104EA000820F911D8F3F910520F4620F60931001D6
:104EB00003C08FEF80931001809110011F928F9398
:104EC00088ED96E09F938F930E94EB070F900F90D1
:104ED0000F900F900895833081F128F4813059F0BC
:104EE0008230D1F00895853009F449C0B8F1863098
:104EF00009F456C0089580911501681720F4861BA7
:104F00008093150102C010921501809115011F9226
:104F10008F9389EC96E054C080911401681720F4B7
:104F2000861B8093140102C0109214018091140119
:104F30001F928F9387EB96E043C08091130168170F
:104F400020F4861B8093130102C0109213018091FC
:104F500013011F928F9384EA96E032C08091120170
:104F6000681720F4861B8093120102C01092120170
:104F7000809112011F928F938FE896E021C080915B
:104F80001101681720F4861B8093110102C0109252
:104F90001101809111011F928F9386E796E010C056
:104FA00080911001681720F4861B8093100102C0C5
:104FB00010921001809110011F928F938BE596E063
:104FC0009F938F930E94EB070F900F900F900F907D
:104FD0000895CF93C82F1F928F9320E639E03F9317
:104FE0002F930E94EB0761E070E080E090E004C046
:104FF000660F771F881F991FCA95D2F70E949C1EC3
:105000000F900F900F900F90CF910C94A01ACF9308
:105010008D3109F465C0B0F58E3009F4CBC100F5CF
:10502000873009F49BC1A8F4863009F06AC28091E8
:10503000D701817F8E7F8093D70185E699E00E941A
:10504000520781EA9DE00E94520781E08093E701C8
:1050500080C1883009F44FC08B3009F47CC151C243
:10506000863109F4EDC138F4803109F4B6C18131DB
:1050700009F42DC246C2893109F4CBC18B3109F440
:1050800086C13FC2853309F434C248F4873209F43B
:1050900030C208F430C2893209F42BC232C28334E0
:1050A00038F48A3308F029C2883309F454C129C27C
:1050B000833409F41EC2883409F023C20E94A01A66
:1050C00080E99DE00E9452079FEF23ED80E391501D
:1050D00020408040E1F700C000000E94332239C127
:1050E00080EB9DE00E9452070E94002C0E94DB147E
:1050F0000E94190D2EC185EA9DE00E94520786E7A5
:105100009BE00E9452070E94F7231F928F9383E730
:105110009BE09F938F930E94EB0781E79BE00E94A7
:1051200052070E94EE23C82F8EE59BE00E94520793
:105130001F92CF9329E53BE03F932F930E94EB070B
:1051400087E59BE00E9452078DE49BE00E94520796
:105150008C2F81701F928F932AE43BE03F932F9313
:105160000E94EB0788E49BE00E9452078EE39BE0DD
:105170000E945207C1FB882780F91F928F932BE36F
:105180003BE03F932F930E94EB0789E39BE00E9453
:1051900052078DE29BE00E945207C2FB882780F9EC
:1051A0001F928F932AE23BE03F932F930E94EB07DD
:1051B00088E29BE00E9452078FE19BE00E94520729
:1051C000C3FBCC27C0F91F92CF938CE19BE09F9348
:1051D0008F930E94EB078AE19BE00E9452070E9496
:1051E0000024C82F86E09BE00E9452071F92CF93B5
:1051F00021E03BE03F932F930E94EB078FEF9AE073
:105200000E94520786EE9AE00E9452078C2F81700E
:105210001F928F9323EE3AE03F932F930E94EB0768
:105220008DB79EB780960FB6F8949EBF0FBE8DBF08
:1052300081EE9AE00E9452078AEC9AE00E9452079F
:10524000C1FB882780F91F928F9327EC3AE03F93A8
:105250002F930E94EB0785EC9AE00E94520783EBA4
:105260009AE00E945207C2FB882780F91F928F9311
:1052700020EB3AE03F932F930E94EB078EEA9AE0EF
:105280000E9452078CE99AE00E945207C3FB8827CC
:1052900080F91F928F9329E93AE03F932F930E9460
:1052A000EB0787E99AE00E9452078DE89AE00E9496
:1052B0005207C4FB882780F91F928F932AE83AE0AF
:1052C0003F932F930E94EB0788E89AE00E945207D1
:1052D00086E79AE00E945207C5FB882780F91F9253
:1052E0008F9323E73AE03F932F930E94EB0781E7E8
:1052F0009AE00E94520785E59AE00E945207C6FB99
:10530000882780F91F928F9322E53AE03F932F93ED
:105310000E94EB0780E59AE00E94520788E49AE039
:105320000E945207C7FBCC27C0F91F92CF9385E498
:105330009AE09F938F930E94EB0783E49AE00E9488
:1053400052078DB79EB74C960FB6F8949EBF0FBE0E
:105350008DBFC1E0DBC08CE899E058C08091D701D7
:10536000C82FC17080FF09C083E89DE00E945207EA
:105370008091D701817F8E7F44C087E79DE00E94A6
:1053800052078091D70181608093D701E2CF80914D
:10539000D70181FBCC27C0F991E0C927C0FB81F977
:1053A0008093D701CC2319F08AE69DE025C08CE5D7
:1053B0009DE02CC08091D70182FBCC27C0F991E001
:1053C000C927C0FB82F98093D701CC2319F08DE463
:1053D0009DE012C08DE39DE019C08091D70183FB51
:1053E000CC27C0F991E0C927C0FB83F98093D7018E
:1053F000CC2351F081E39DE00E9452078091D701B8
:1054000081608093D70182C084E29DE00E945207B0
:10541000A0CF85E19DE00E94520789EE9CE00E94AA
:1054200052078CEA9CE00E94520785E89CE00E94AB
:10543000520781E49CE00E94520786E19CE0E6CF9F
:1054400088E09CE00E9452070E94DB141F928F9319
:105450008EEE9BE09F938F930E94EB0780910C014F
:105460001F928F9387ED9BE09F938F930E94EB0792
:1054700080916E011F928F9384EC9BE09F938F939A
:105480000E94EB0780910D011F928F9381EB9BE0AF
:105490009F938F930E94EB078091D9019091DA013D
:1054A000A091DB01B091DC01BF93AF939F938F93E9
:1054B0008DE99BE09F938F930E94EB078DB79EB77A
:1054C00046960FB6F8949EBF0FBE8DBF42CF0E9486
:1054D000A01AC0910D0181E0C827C0930D01CC2313
:1054E00029F083E99BE00E94520710C088E89BE006
:1054F0008DCF80E003C08D5101C089530E94E92700
:1055000028CF86E89BE00E945207C0E08C2FCF9105
:10551000089580E0089580E00895CF93C82F80918A
:10552000E701813081F020F0823009F44CC042C1A3
:10553000A0910E01B0910F018C91813169F08232FE
:1055400009F03AC109C0A0910E01B0910F018C91F0
:10555000813111F0823249F48C2F0E94892A811105
:105560002FC08C2F0E9407282CC08C2F0E948B2AC2
:10557000811126C0C431E1F070F4CB3081F0C0312C
:10558000D1F40E94B12688E599E00E94520782E09A
:105590008093E70115C0C93259F0C83361F485E63C
:1055A00099E00E9452078CE599E00E94520708C0DA
:1055B0001092E70103C186E599E00E945207FEC000
:1055C00081E08170FDC0C43220F5CE3108F0C0C04A
:1055D000CB3099F1C8F4C73009F0D2C08AE080938B
:1055E000150194E19093140193E09093130180933B
:1055F000120188E08093110188E2809310018CEF02
:1056000097E00E945207BFC0C33149F1C431C1F0D5
:10561000B7C0CB3409F4A9C028F4C93289F0C83323
:1056200061F0AEC0C13509F49EC0C23509F499C01D
:10563000CE3409F0A5C06AE09EC00E94B126A3C086
:105640008091E601882319F01092E6019CC089E060
:1056500098E00E94520781E08093E701B1C083EE99
:1056600097E00E94520781ED97E00E9452078091D7
:1056700015011F928F938EEC97E09F938F930E945A
:10568000EB078CEC97E00E9452078AEB97E00E94B0
:105690005207809114011F928F9387EB97E09F939D
:1056A0008F930E94EB0785EB97E00E94520786EAF2
:1056B00097E00E945207809113011F928F9383EA13
:1056C00097E09F938F930E94EB0781EA97E00E94F7
:1056D000520780E997E00E945207809112011F92C1
:1056E0008F938DE897E09F938F930E94EB078BE851
:1056F00097E00E94520786E797E00E945207809148
:1057000011011F928F9383E797E09F938F930E94DD
:10571000EB0781E797E00E9452078AE597E00E9435
:105720005207809110011F928F9387E597E09F9316
:105730008F930E94EB0785E597E00E9452078DB793
:105740009EB748960FB6F8949EBF0FBE8DBF1BC084
:10575000CE51EC2FF0E0E15DFE4F80818093E601B9
:1057600012C061E003C061E006C06AE08091E6011A
:105770000E94C82608C08091E6010E946B2703C0E2
:105780008AEF97E013C08091E601882369F01F92A9
:105790008F9384EF97E09F938F930E94EB070F9076
:1057A0000F900F900F9004C081EF97E00E94520776
:1057B00081E006C01092E70180E002C080E001CFE6
:1057C000CF910895E1E8F0E0808188608083808156
:1057D000816080838FB7F89493E09093890090ED77
:1057E000909388008FBF0895EFE6F0E0808182609B
:1057F00080830895EFE6F0E080818D7F80830895B7
:10580000EFE6F0E0808192E08927808308951F927F
:105810000F920FB60F9211242F933F934F935F93E4
:105820006F937F938F939F93AF93BF93EF93FF9368
:105830008091E8019091E90101969093E9018093AC
:10584000E801811103C082E00E94190DE091E90195
:10585000E695E695F0E0E054F24FE4918091E8019E
:105860008E1303C080E00E94190DFF91EF91BF914C
:10587000AF919F918F917F916F915F914F913F91E8
:105880002F910F900FBE0F901F90189504D0689421
:10589000B1118DC0089570D088F09F5790F0B92F46
:1058A0009927B751A0F0D1F0660F771F881F991F75
:1058B0001AF0BA95C9F712C0B13081F077D0B1E0D3
:1058C000089574C0672F782F8827B85F39F0B93FE3
:1058D000CCF3869577956795B395D9F73EF4909577
:1058E0008095709561957F4F8F4F9F4F0895E894F5
:1058F00009C097FB3EF490958095709561957F4F18
:105900008F4F9F4F9923A9F0F92F96E9BB279395C5
:10591000F695879577956795B795F111F8CFFAF4D5
:10592000BB0F11F460FF1BC06F5F7F4F8F4F9F4F06
:1059300016C0882311F096E911C0772321F09EE864
:10594000872F762F05C0662371F096E8862F70E0CA
:1059500060E02AF09A95660F771F881FDAF7880FA4
:105960009695879597F9089557FD9058440F551FC0
:1059700059F05F3F71F04795880F97FB991F61F0D1
:105980009F3F79F087950895121613061406551F48
:10599000F2CF4695F1DF08C0161617061806991FB4
:1059A000F1CF86957105610508940895E894BB27A9
:1059B00066277727CB0197F908950BD078C069D077
:1059C00028F06ED018F0952309F05AC05FC011245A
:1059D000EECFCADFA0F3959FD1F3950F50E0551F8E
:1059E000629FF001729FBB27F00DB11D639FAA2734
:1059F000F00DB11DAA1F649F6627B00DA11D661F83
:105A0000829F2227B00DA11D621F739FB00DA11DA3
:105A1000621F839FA00D611D221F749F3327A00D5D
:105A2000611D231F849F600D211D822F762F6A2FF9
:105A300011249F5750408AF0E1F088234AF0EE0F7E
:105A4000FF1FBB1F661F771F881F91505040A9F78B
:105A50009E3F510570F014C0AACF5F3FECF3983E13
:105A6000DCF3869577956795B795F795E7959F5FF2
:105A7000C1F7FE2B880F911D9695879597F908958C
:105A800097F99F6780E870E060E008959FEF80ECF1
:105A9000089500240A941616170618060906089594
:105AA00000240A9412161306140605060895092EFA
:105AB0000394000C11F4882352F0BB0F40F4BF2B69
:105AC00011F460FF04C06F5F7F4F8F4F9F4F0895A9
:105AD000991B79E004C0991F961708F0961B881F40
:105AE0007A95C9F78095089597FB072E16F40094D0
:105AF00007D077FD09D00E948E2D07FC05D03EF41B
:105B0000909581959F4F0895709561957F4F089569
:105B1000EE0FFF1F0590F491E02D0994AA1BBB1B0B
:105B200051E107C0AA1FBB1FA617B70710F0A61B9D
:105B3000B70B881F991F5A95A9F780959095BC01BE
:105B4000CD010895F999FECF92BD81BDF89A9927AC
:105B500080B50895A8E1B0E042E050E00C94C52D76
:105B6000262FF999FECF1FBA92BD81BD20BD0FB679
:105B7000F894FA9AF99A0FBE019608950E94B02DF2
:105B8000272F0C94B12DDC01CB01FC01F999FECF3C
:105B900006C0F2BDE1BDF89A319600B40D924150B5
:0A5BA0005040B8F70895F894FFCFC5
:105BAA0020021A0D0B0EE80DB40D810D0101C5017D
:105BBA0028080A03140A3F4D3620394605F904C35A
:105BCA0004A3046A04DD03F6030F0428044804014D
:0A5BDA000203040506070809000095
:00000001FF
